:1000000024C0189518951895189535C01895189509
:1000100018951895189546616872747265676C65D5
:1000200072204156522039305332333133205665D5
:100030007273696F6E20302E3120546573745C309A
:1000400030305C3030305C3030300FED0DBF00E0D0
:100050000FBD03E00EBD0CED0CBD0BE00DBD00E8C7
:1000600009BF78940FEF07BB01BB789430E0089488
:1000700038BB32BBFDCF331F0CED0CBD0BE00DBD0B
:020080001895D1
:00000001FF
